:100000000C94FC030C9440040C9440040C944004A5
:100010000C9440040C9440040C9440040C94400450
:100020000C9440040C9440040C940E0F0C94E00FBC
:100030000C9440040C9440040C9440040C94400430
:100040000C9440040C94AA240C9440040C94400496
:100050000C9440040C94391E0C9440040C944004FD
:100060000C9440040C9440040C9440040C94400400
:100070000C9440040C9440040C9440040C944004F0
:100080000C9440040C9440040C9440040C944004E0
:100090000C9440040C9440040C9440040C944004D0
:1000A0000C9440040C9440040C944004FF046A0433
:1000B0001605B804C904E7048204AC04B204A6041B
:1000C000E104BD04C3049A04A00450044D106F1051
:1000D0005D116F105D11B410D7105D112C113F111F
:1000E0002B142B1468146814AB14E91402170217AC
:1000F0000215021703160316D61602170217ED167D
:1001000002E002E2012E022E02E10002E002E10220
:10011000E20001E001E101E20002E001E301190275
:100120001902E30002E00001E00002E002E30164E2
:1001300002640002E002E30001E001E30001E101EA
:1001400037023702E10138023801E10125022502B8
:10015000E10002E002E1013102310002E002E100CF
:1001600001E001E10001E10137023702E10138025B
:100170003801E10107020702E100013502350120E3
:1001800002200002E302E10001E301E10001E101DC
:1001900036023602E10138023801E1012602260268
:1001A000E10001E10137023702E10138023801E1E3
:1001B0000126022602E10001E10136023602E101D8
:1001C00038023801E10125022502E10001E1013791
:1001D000023702E10138023801E20125022502E27C
:1001E0000001E10137023702E10138023801E10183
:1001F00030023002E10002E002E20130023000028F
:10020000E002E20001E001E20002E001E301060297
:100210000602E30002E00001E00029002B00E200FA
:10022000E100358100001E00140004001D7105303E
:100230004D831F001A0016001B0006304C002000E2
:1002400008000700060052002A00210015000900DE
:10025000190051004A00220017000A0005000000A2
:1002600002300430E3000000E200000002540430D9
:10027000E7000000E6000000045423001C000B000F
:10028000110000002E7F240018000D001000500007
:100290004B0025000C000E0036004F002C002600FD
:1002A00012000F003700E108280027001300330078
:1002B0003871E1044E002D002F003474E5003081C8
:1002C00000000100010001000100010000003A00EF
:1002D000350031000100010001003B003502210220
:1002E000350001004C003C001E02240622020100E1
:1002F00001003D002D0224022404010001003E0003
:10030000010037001104000001000100010000009D
:100310000100000001000F3001000000010000009A
:1003200068003F0024062402240400004500400029
:10033000220425021104310269004100230426022F
:1003400064005000010042003500250452005100B5
:10035000010043003502260438004F006A004400C3
:100360001E02310021020100000001000100010015
:100370000100010000000100010001000100010076
:1003800001000100F400F200FB0001000100010087
:10039000F000F100FA00010001000100F500F30097
:1003A000FC00010001000100F900FA00F600000065
:1003B0000100010001000000010000000100A80090
:1003C0000100000001000000010001000100A9007F
:1003D000AA0000000100010001000100010001006D
:1003E0000100010001000100AC000100B6000100A5
:1003F00001000100AB0050000100010001000100FC
:10040000520051000100AE000100010001004F0048
:1004100000000100010001000100010000000100D6
:1004200001000100010001000100010001000100C4
:1004300001000100010001000100010001000100B4
:1004400001000100010001000100010001000100A4
:100450000100010001000000010001000100000096
:100460000100000001000730010000000100000051
:10047000010008300E300B300100000001000C308C
:100480000A300D30010001000100010009300100B7
:100490000100010001000100010001000100010054
:1004A0000100010001000100010001000100010044
:1004B0000100010001000100000001000100010035
:1004C0000100010000000100010001000100010025
:1004D00001000100010050000100010001000100C5
:1004E00052005100010001000100010001004F0015
:1004F00001000100010001000100010001000000F5
:1005000001000100010000000100000001000100E5
:10051000010000000100000001003F0052005100F6
:100520002302000001004000240021001E002700DB
:1005300001004100250022001F0037000100420099
:100540002600230020003600010043003002300066
:100550002402270201004400450038000100010088
:10056000000001000100E1000100E00000000100C6
:1005700001000100010001003D0001000100010037
:1005800001000100E0000100010001000100010084
:100590002C00010001000100010001003C000100ED
:1005A00001000100010000003A000100010000000C
:1005B000010000003B000F300100000001000000BE
:1005C0000100010001000100010000000100010024
:1005D0000100010001000100010001000100010013
:1005E0000100010001000100010001000100010003
:1005F00001000100010001000100010001000100F3
:100600000100010001000100000016034500720016
:1006100067006F0044006F007800200045005A001A
:10062000000016034500720067006F0044006F0071
:100630007800200045005A00000004030904090264
:100640006D00040100A0FA0904000001030101008B
:10065000092111010001223F000705810308000A5A
:100660000904010001030102000921110100012216
:100670004D000705820308000A0904020001030077
:10068000000009211101000122360007058303083B
:10069000000A090403000103000000092111010000
:1006A0000122390007058403100001120110010026
:1006B000000008EDFE071301000102000105010919
:1006C00006A101050719E029E71500250195087520
:1006D0000181020508190129059505750191029509
:1006E000017503910105071900297715002501956A
:1006F0007875018102C005010980A10185021601FA
:100700000026B7001A01002AB70075109501810074
:10071000C0050C0901A1018503160100269C021ADF
:1007200001002A9C02751095018100C00501090293
:10073000A1010901A10005091901290515002501DB
:100740009505750181029501750381010501093047
:1007500009311581257F95027508810609381581B3
:10076000257F950175088106050C0A38021581253B
:100770007F950175088106C0C005010906A1010524
:100780000719E029E71500250195087501810295F3
:100790000175088101050819012905950575019163
:1007A000029501750391010507190029FF15002520
:1007B000FF950675088100C00000000000000000E1
:1007C000000000010204060A0F17202C3A4A5D714E
:1007D000879DB3C7DAE9F5FCFFFCF5E9DAC7B39DFD
:1007E00087715D4A3A2C20170F0A060402010000A7
:1007F000000000000000000011241FBECFEFDAE06F
:10080000DEBFCDBF04B603FE24C08091F0019091FD
:10081000F101A091F201B091F3018730904BA74014
:10082000B04BB9F41092F0011092F1011092F20164
:100830001092F30114BE84B7877F84BF88E10FB69E
:10084000F89480936000109260000FBEE0E0FFE338
:10085000099511E0A0E0B1E0E8EDFCE402C00590EC
:100860000D92A433B107D9F711E0A4E3B1E001C0C0
:100870001D92A03FB107E1F70E94520C0C946A262A
:100880000C940000462F50E04031510508F0F1C0B3
:10089000DC01FA01EA5AFF4F12968C910C941F2644
:1008A000882309F4E6C08091B3019091B401A0912E
:1008B000B501B091B60120E2822780729927AA275C
:1008C000BB278093B3019093B401A093B501B0937B
:1008D000B601CFC0882349F00E94031E90933501D2
:1008E0008093340187E192E00895809134019091E2
:1008F00035010E940F1E873991050CF0AEC089E0CA
:1009000092E00895882349F00E94031E90933501D8
:100910008093340184E092E00895809134019091B5
:1009200035010E940F1E873991050CF099C086EFA2
:1009300091E00895882309F49CC081EE91E0089528
:10094000882309F496C08CEC91E00895882309F47B
:1009500090C087EB91E00895882309F48AC082EA69
:1009600091E00895882309F484C08DE891E008950A
:10097000811179C083E891E00895882309F479C052
:100980008AE791E00895882309F473C085E691E031
:100990000895882349F00E94031E909335018093A7
:1009A000340180E691E00895809134019091350101
:1009B0000E940F1E873991050CF058C082E591E026
:1009C0000895882309F455C08DE391E008958823A4
:1009D00049F00E94031E909335018093340188E30F
:1009E00091E0089580913401909135010E940F1E8D
:1009F000873991050CF040C08AE291E00895882380
:100A000049F00E94031E909335018093340187E2E0
:100A100091E0089580913401909135010E940F1E5C
:100A20008739910564F589E191E00895882349F0BB
:100A30000E94031E909335018093340182E191E07E
:100A4000089580913401909135010E940F1E8739DD
:100A50009105C4F480E091E0089584E192E0089566
:100A60008FEF91E0089588E891E008958BE591E09B
:100A7000089580E090E0089583E391E0089584E292
:100A800091E008958BE091E0089508956091B3019D
:100A90007091B4018091B5019091B6010E94651DDD
:100AA00056985E9825982D9826982E9827982F98D6
:100AB0008330C1F028F4813041F0823049F008954C
:100AC000843049F0853051F00895259A2D9A089583
:100AD000269A2E9A0895259A2D9A04C0259A2D9A21
:100AE000269A2E9A279A2F9A08950C94460556987E
:100AF0005E9825982D9826982E9827982F988FEFF6
:100B000090E0909389008093880090938B0080936D
:100B10008A0090938D0080938C00259A2D9A2FEF58
:100B200080E792E0215080409040E1F700C0000053
:100B3000269A2E9A2FEF80E792E021508040904035
:100B4000E1F700C00000279A2F9A2FEF80E792E08C
:100B5000215080409040E1F700C0000025982D987A
:100B60002FEF80E792E0215080409040E1F700C0F5
:100B7000000026982E982FEF80E792E021508040C9
:100B80009040E1F700C0000027982F9856985E9893
:100B900025982D9826982E9827982F98089589EAB9
:100BA0008093800089E08093810024982C983F985E
:100BB0008AB18F748AB96E98479A8BB1806B8BB962
:100BC000769A0E9477050C94450580E28093000197
:100BD0008091360181110EC00E94340681E080931D
:100BE00036012FEF83ED90E3215080409040E1F7F4
:100BF00000C0000080E40E943A0680930001811149
:100C00002EC00E94640680930001811128C00E94BA
:100C1000640680930001811122C08FE30E94640664
:100C20008093000181111BC00E945C0680E40E9439
:100C30003A0680930001811112C08CE00E94640684
:100C40008093000181110BC00E9464068093000113
:100C5000811105C08FE30E946406809300010E9409
:100C60005C068091000108951092B9008AE080939B
:100C7000B800089594EA9093BC009091BC0097FF4F
:100C8000FCCF9091B900987F983021F0903111F00D
:100C900081E008958093BB0084E88093BC0080913C
:100CA000BC0087FFFCCF8091B900887F883111F0AC
:100CB000803471F780E0089584E98093BC008091CE
:100CC000BC0084FDFCCF08958093BB0084E8809332
:100CD000BC008091BC0087FFFCCF9091B900987F49
:100CE00081E0983209F480E0089584E88093BC00A4
:100CF0008091BC0087FFFCCF8091BB00089580915C
:100D00000001811115C080E40E943A068093000121
:100D100081110CC082E10E94640680930001811160
:100D200005C08FEF0E946406809300010E945C065C
:100D300084B1807F84B985B1807F85B98AB1837F92
:100D40008AB98BB1837F8BB93E98469808950E94EB
:100D5000E505809300010E947F0680B38C7080BB04
:100D600081B3836F81BBA8E3B1E0E6E4F1E08EE0FC
:100D70008E0F11921D928E13FCCF0C94CF05BF9253
:100D8000CF92DF92EF92FF920F931F93CF93DF9357
:100D900080910001882379F0809137018F5F8093E3
:100DA0003701811108C00E94E5058093000181117F
:100DB00002C00E94770508E311E0C0E0D0E0DD2426
:100DC000D39482E0C82EEE24E394F12CC730D105F1
:100DD00000F580910001811164C080E40E943A0610
:100DE00080930001811112C082E10E946406809309
:100DF000000181110BC0C7010C2E01C0880F0A949D
:100E0000EAF780950E946406809300010E945C06C8
:100E100048C0CA30A1F028F4C83059F0C93061F098
:100E200005C0CC3089F070F0CD3089F0209A289838
:100E300010C0219A29980DC0229A2A980AC0239A94
:100E40002B9807C0529A01C0539A5B9802C03E9AF1
:100E5000469890EA9A95F1F79FB1799902C082E09D
:100E600001C080E091709D25982B7C9902C084E0A0
:100E700001C080E0892B7D9902C038E001C030E0DC
:100E8000832B7E9902C020E101C020E0822B9FB11C
:100E90009095991F9927991F9295990F907E892B6C
:100EA0000FC080910001811149C080E40E943A0680
:100EB00080930001882379F1B12C0E945C068B2D70
:100EC000F8019081981719F08083C09201010E9467
:100ED0007F0621960F5F1F4FCE30D10509F076CFE8
:100EE00080910101882361F1815080930101882361
:100EF00039F08FE99FE00197F1F700C0000020C0B2
:100F0000A6E4B1E0E8E3F1E0CF01825F91919D9327
:100F10008E13FCCF15C083E10E946406809300010C
:100F20008111CACF81E40E943A06809300018111A9
:100F3000C3CF0E947506B82EB094BFCF80E0C0CF5B
:100F40000E94750581E0DF91CF911F910F91FF9075
:100F5000EF90DF90CF90BF900895E82FF0E0EA5B2C
:100F6000FE4F808108950895089596E0799FF001DD
:100F7000112494E5899FE00DF11D1124E60FF11D68
:100F8000EE0FFF1FE65EFD4F859194910895880F47
:100F9000991FFC01E656FF4F859194910895880FA3
:100FA000991FFC01E65EFD4F8591949108950F9382
:100FB0001F93CF93DF93EC018115904350F5C1153A
:100FC00080E2D80708F0B3C0CB3BD10590F4C83A13
:100FD000D10508F05AC0C53AD10508F04BC0C4305D
:100FE000D10508F0BBC1219709F0B5C101E010E0BF
:100FF000F5C1CF3FD10511F008F0B0C1C03FD10518
:1010000008F092C0CE01805E9109089708F4A6C14D
:10101000A2C1C11591E5D907A8F4C23020E5D207D5
:1010200008F09EC0C11580E5D80709F485C008F016
:1010300091C0C11520E4D20708F08DC1DD278E01D3
:10104000106CCCC1C11580E8D80758F4C11590E7E1
:10105000D90708F07CC1C11520E6D20708F422C1E7
:101060007AC1C11580E9D80708F075C1DF708E011B
:10107000106AB4C1C53AD10509F472C1C63AD105A6
:1010800009F071C102E810E4A9C1C83AD10509F418
:101090006DC1C93AD10509F46CC1CA3AD10509F448
:1010A0006BC1CB3AD10509F46AC1CC3AD10509F438
:1010B00069C1CD3AD10509F468C1C03BD10509F435
:1010C00067C1CE3AD10509F466C1CF3AD10509F41A
:1010D00065C1C13BD10509F464C1C23BD10509F426
:1010E00063C1C33BD10509F462C1C43BD10509F416
:1010F00061C1C53BD10509F460C1C63BD10509F406
:101100005FC1C73BD10509F45EC1C83BD10509F4F5
:101110005DC1C93BD10509F45CC1CA3BD10509F4E5
:101120005BC100E014E45AC18E01106557C1CE01C5
:101130009F700E94CF0753C10E9426179FEF24E3A0
:101140008CE0915020408040E1F700C000000E94F8
:101150005E1E44C18091CF0181608093CF013EC16A
:101160000E940720811102C00E94ED1F0E942420CE
:1011700090E09093F0018093EF01C23090E5D907A1
:1011800021F48091EF01816086C0C43020E5D20750
:1011900021F48091EF0182607EC0C63080E5D807DF
:1011A00021F48091EF01846076C0C83090E5D907C2
:1011B00019F48091EF0127C0CA3020E5D20721F44D
:1011C0008091EF01806167C0CC3080E5D80721F4C1
:1011D0008091EF0180625FC0CE3090E5D90721F4A5
:1011E0008091EF01806457C0C03120E5D20721F41F
:1011F0008091EF0180684FC0C23180E5D80729F4A3
:101200008091EF018460886046C0C33090E5D907C3
:1012100021F48091EF018E7F3EC0C53020E5D207DA
:1012200021F48091EF018D7F36C0C73080E5D8076B
:1012300021F48091EF018B7F2EC0C93090E5D90752
:1012400019F48091EF0126C0CB3020E5D20721F4BC
:101250008091EF018F7E1FC0CD3080E5D80721F44B
:101260008091EF018F7D17C0CF3090E5D90721F431
:101270008091EF018F7B0FC0C13120E5D20721F4AF
:101280008091EF018F7707C0C331D04531F4809151
:10129000EF018B7F877F8093EF018091EF010E94A8
:1012A00028209CC08D2F99278F7099278130910518
:1012B000D9F49E012370332702C0880F991F2A9505
:1012C000E2F79C688E0144E0000F111F4A95E1F798
:1012D00000271370802B912B53E0CC0FDD1F5A9504
:1012E000E1F7C076DD272FC08230910531F4DC2F85
:1012F000CC278E01016F106A71C08330910569F4AB
:10130000CE018370992701E010E002C0000F111F89
:101310008A95E2F7C8019C680FC0049709F05EC087
:10132000CE018370992701E010E002C0000F111F69
:101330008A95E2F7C8019A6823E0CC0FDD1F2A9551
:10134000E1F7C07ED7708C010C2B1D2B47C0DF70DE
:101350008E01106243C000E010E040C08E013EC02C
:1013600001E810E43BC003E810E438C002EE14E4E6
:1013700035C009EE14E432C00AEE14E42FC005EBC8
:1013800014E42CC006EB14E429C007EB14E426C0D7
:101390000CEC14E423C00DEC14E420C003E815E4C5
:1013A0001DC00AE815E41AC002E915E417C004E9F3
:1013B00015E414C001E216E411C003E216E40EC005
:1013C00004E216E40BC005E216E408C006E216E4E7
:1013D00005C007E216E402C00AE216E4C801DF9184
:1013E000CF911F910F91089596E0799FF0011124FC
:1013F00094E5899FE00DF11D1124E60FF11DEE0F1C
:10140000FF1FE65EFD4F85919491803E9105E0F4CB
:10141000803C910558F58133910509F46FC048F47B
:101420008932910509F463C08A32910509F46DC0CF
:1014300072C089339105E9F082389105D1F0853386
:10144000910509F44DC067C0833E910581F138F4E0
:10145000803E9105B9F0823E9105D9F05CC0863E90
:10146000910561F1873E9105A1F155C00E94C70722
:1014700008952091EF0120FD02C021FF4CC080EEB5
:1014800090E049C08091EF0180FFF9CF89E390E0BF
:1014900042C08091EF0182FF0EC08091EF0184FF76
:1014A00003C080E090E037C083EE90E034C08091CC
:1014B000EF0182FFF2CF82EE90E02DC08091EF012C
:1014C00083FF0BC08091EF0184FDEBCF87EE90E0AE
:1014D00022C08091EF0183FFF5CF86EE90E01BC024
:1014E0008091EF0185FF07C089E290E014C08091F0
:1014F000EF0185FFF9CF85E390E00DC08091EF010A
:1015000086FF07C08AE290E006C08091EF0186FF67
:10151000F9CF81E390E00E94D707089508950C94D5
:101520008E0A809164010895CF93DF9300D01F92BB
:10153000CDB7DEB79C018091E601843019F593E0C8
:1015400099833B832A839093E9008FEF9091E80081
:10155000815095FD06C095ED9A95F1F70000811137
:10156000F5CF8091E80085FF0DC040E050E063E0DA
:1015700070E0CE0101960E94FE0C8091E8008E770B
:101580008093E8000F900F900F90DF91CF91089516
:10159000CF93DF9300D01F92CDB7DEB72091E60145
:1015A000243021F522E029839B838A8383E0809382
:1015B000E9008FEF9091E800815095FD06C095ED10
:1015C0009A95F1F700008111F5CF8091E80085FF31
:1015D0000DC040E050E063E070E0CE0101960E9453
:1015E000FE0C8091E8008E778093E8000F900F90BA
:1015F0000F90DF91CF9108952091E6012430F1F40E
:1016000022E02093E9002FEF3091E800215035FDD2
:1016100006C035ED3A95F1F700002111F5CF209184
:10162000E80025FF0BC040E050E065E070E00E945C
:10163000FE0C8091E8008E778093E8000895CF93A8
:10164000DF93EC019091E601943009F046C080915F
:101650000C018823D9F080910D018823B9F0909373
:10166000E9008FEF9091E800815095FD06C095E16B
:101670009A95F1F700008111F5CF8091E80085FF80
:101680002CC040E050E060E170E017C081E0809342
:10169000E9008FEF9091E800815095FD06C095ED2F
:1016A0009A95F1F700008111F5CF8091E80085FF50
:1016B00014C040E050E068E070E0CE010E94FE0CF3
:1016C0008091E8008E778093E80080E1FE01A4E538
:1016D000B1E001900D928A95E1F7DF91CF910895E5
:1016E0008091E501811109C00E94930E0E94F00EC5
:1016F0008091E20084608093E20008951092E501F9
:10170000089508950C9497240E94F41D0E949D242E
:101710000E9496110C948F0A42E061EC81E00E94D5
:101720000D0E42E061EC82E00E940D0E42E061ECA1
:1017300083E00E940D0E42E161EC84E00C940D0EFA
:101740008091E801833009F455C030F4813071F0A4
:10175000823009F48EC008958A3009F47AC08B3043
:1017600009F460C0893009F09CC020C08091E70175
:10177000813A09F096C08091E800877F8093E80065
:101780008091EB019091EC01892B21F460E184E5DB
:1017900091E003C060E080E090E070E00E94490DBD
:1017A0008091E8008B778093E80008958091E701AD
:1017B000813209F076C08091EB019091EC010097A5
:1017C00019F0039709F06DC08091E800877F80933E
:1017D000E8008091E80082FD05C08091E60181115A
:1017E000F8CF5FC08091F100809364018091E800A0
:1017F0008B7753C08091E701813A09F052C0809104
:10180000EB019091EC01892B09F04BC08091E8002D
:10181000877F8093E8008091E80080FFFCCF809173
:101820000C0136C08091E7018132D9F58091EB013E
:101830009091EC01892BA9F58091E800877F809336
:10184000E8000E94420E8091E90180930C010C9403
:1018500026178091E701813221F58091E800877F8A
:101860008093E8000E94420E8091EA018093650116
:1018700008958091E701813AA1F48091E800877F83
:101880008093E8008091E80080FFFCCF80916501A3
:101890008093F1008091E8008E778093E8000C94AB
:1018A000420E089584B7877F84BF88E10FB6F8940D
:1018B00080936000109260000FBE90E080E80FB649
:1018C000F89480936100909361000FBE0E94E5112F
:1018D0000E94930E0E94F00E8091E200846080933B
:1018E000E20078940E9476110E94E71182E091E074
:1018F0000E9491110E9485248091E601853069F44F
:101900000E94B51D8091E4018823B1F30E94E01D7F
:10191000882391F30E94E80CEFCF0E94ED11ECCFE9
:10192000292F332723303105C9F064F421303105E4
:1019300081F02230310509F043C08DE690E02EE3BE
:1019400036E042C021323105F1F02232310541F159
:1019500037C082E190E02BEA36E036C0992781302B
:10196000910541F08230910541F0892B49F5EAE378
:10197000F6E005C0E2E2F6E002C0EAE0F6E08491BB
:1019800090E09F0121C06430D8F4E62FF0E0EE0F24
:10199000FF1FEE5DFE4F2081318189E090E014C091
:1019A000643070F470E0FB01EE0FFF1FE65EFE4F47
:1019B00020813181FB01EA5EFE4F808190E004C00E
:1019C00080E090E020E030E0FA0131832083089548
:1019D00080E189BD82E189BD09B400FEFDCF80911F
:1019E000D8008F7D8093D8008091E0008260809342
:1019F000E0008091E00081FDFCCF0895CF92DF925E
:101A0000EF92FF920F931F93CF93DF93EC018B0123
:101A10006A010E94610E811133C0C114D10439F0F2
:101A2000F60180819181081B190BC80FD91FE12C89
:101A3000F12C0115110519F18091E80085FD16C002
:101A40008091E8008E778093E800C114D10449F0BA
:101A5000F60180819181E80EF91EF182E08285E035
:101A60000FC00E94610E882321F30AC089918093E0
:101A7000F10001501109FFEFEF1AFF0ADACF80E001
:101A8000DF91CF911F910F91FF90EF90DF90CF905A
:101A900008952091ED013091EE012617370748F0A7
:101AA0006115710539F42091E8002E772093E80044
:101AB00001C0B90140E061157105A9F12091E6016D
:101AC000222309F443C0253009F442C02091E800E4
:101AD00023FD40C02091E80022FD32C02091E800A3
:101AE00020FFE9CF4091F3002091F20030E0342B49
:101AF000FC01CF016115710559F02830310540F422
:101B000081918093F100615071092F5F3F4FF1CFB8
:101B100041E02830310509F040E02091E8002E77BF
:101B20002093E800C8CF4111C9CF0AC08091E601D7
:101B3000882361F0853061F08091E80083FD0AC060
:101B40008091E80082FFF2CF80E0089582E008955E
:101B500083E0089581E008952091ED013091EE0138
:101B60002617370748F06115710539F42091E80010
:101B70002E772093E80001C0B901FC0120E0611537
:101B8000710591F18091E601882309F440C0853008
:101B900009F43FC08091E80083FD3DC08091E800DA
:101BA00082FD2FC08091E80080FFE9CF2091F300F3
:101BB0008091F20090E0922B6115710559F0883008
:101BC000910540F424912093F10031966150710900
:101BD0000196F2CF21E0089709F020E08091E8001B
:101BE0008E778093E800CBCF2111CCCF0AC08091B3
:101BF000E601882361F0853061F08091E80083FD83
:101C00000AC08091E80082FFF2CF80E0089582E070
:101C1000089583E0089581E00895982F973058F54E
:101C20009093E900981739F07091EC002091ED0045
:101C30005091F00003C0242F762F50E021FF19C0EF
:101C40003091EB003E7F3093EB003091ED003D7F13
:101C50003093ED003091EB0031603093EB007093E6
:101C6000EC002093ED005093F0002091EE0027FF50
:101C700007C09F5FD3CF8F708093E90081E0089504
:101C800080E008958091E70187FF11C08091E8000E
:101C900082FD05C08091E6018111F8CF11C08091CD
:101CA000E8008B770BC08091E601882349F0809192
:101CB000E80080FFF8CF8091E8008E778093E800FD
:101CC00008952091E4003091E50095E64091EC0004
:101CD000842F817040FF22C08091E80080FD1CC0ED
:101CE0008091E601882391F0853091F08091EB009E
:101CF00085FD10C04091E4005091E5004217530764
:101D000029F39A01915011F784E0089582E0089533
:101D100083E0089581E0089580E008954091E8000F
:101D200042FFDECF08950E94010F0E94090FE0EEEE
:101D3000F0E0808181608083E8EDF0E080818F7742
:101D4000808319BCA7EDB0E08C918E7F8C9380814D
:101D50008F7E80831092E50108950F931F93CF9398
:101D6000DF930E94010F0E94090FC8EDD0E0888127
:101D70008F77888388818068888388818F7D888336
:101D800019BC1092E6011092E2011092E401109247
:101D9000E30100EE10E0F80180818B7F8083888171
:101DA0008160888342E060E080E00E940D0EE1EEF9
:101DB000F0E080818E7F8083E2EEF0E080818160C0
:101DC0008083808188608083F80180818E7F80831A
:101DD000888180618883DF91CF911F910F91089551
:101DE000E8EDF0E080818F7E8083E7EDF0E0808198
:101DF0008160808384E082BF81E08093E5010C9460
:101E0000AD0EE8EDF0E080818E7F80831092E200DD
:101E100008951092DA001092E10008951F920F9237
:101E20000FB60F9211242F933F934F935F936F93AD
:101E30007F938F939F93AF93BF93EF93FF93809183
:101E4000E10082FF0BC08091E20082FF07C0809119
:101E5000E1008B7F8093E1000E9475118091DA0090
:101E600080FF1FC08091D80080FF1BC08091DA00E6
:101E70008E7F8093DA008091D90080FF0DC080E1D1
:101E800089BD82E189BD09B400FEFDCF81E0809368
:101E9000E6010E94700B05C019BC1092E6010E9479
:101EA0007E0B8091E10080FF19C08091E20080FFED
:101EB00015C08091E2008E7F8093E2008091E20065
:101EC00080618093E2008091D80080628093D80086
:101ED00019BC85E08093E6010E94820B8091E100AD
:101EE00084FF30C08091E20084FF2CC080E189BD76
:101EF00082E189BD09B400FEFDCF8091D8008F7DBD
:101F00008093D8008091E1008F7E8093E1008091E2
:101F1000E2008F7E8093E2008091E20081608093F6
:101F2000E2008091E201882311F084E007C08091F3
:101F3000E30087FD02C081E001C083E08093E601F9
:101F40000E94840B8091E10083FF29C08091E20010
:101F500083FF25C08091E100877F8093E10082E0CC
:101F60008093E6011092E2018091E1008E7F8093E0
:101F7000E1008091E2008E7F8093E2008091E20098
:101F800080618093E20042E060E080E00E940D0EFC
:101F90008091F00088608093F0000E94810BFF9197
:101FA000EF91BF91AF919F918F917F916F915F91D1
:101FB0004F913F912F910F900FBE0F901F9018954A
:101FC0001F920F920FB60F9211242F933F934F93AE
:101FD0005F936F937F938F939F93AF93BF93CF93B1
:101FE000DF93EF93FF93C091E900CF708091EC00F5
:101FF000D82FD17080FDD0E81092E9008091F000D8
:10200000877F8093F00078940E9424101092E9005A
:102010008091F00088608093F000CD2BCF70C0934A
:10202000E900FF91EF91DF91CF91BF91AF919F9127
:102030008F917F916F915F914F913F912F910F9071
:102040000FBE0F901F9018951F93CF93DF93CDB7BE
:10205000DEB7AA970FB6F894DEBF0FBECDBFE7EE8E
:10206000F1E088E08E0F9091F10091938E13FBCFF9
:102070000E94A00B8091E80083FF1FC18091E701BF
:102080009091E801492F50E04A30510508F015C100
:10209000FA01EA59FF4F0C941F26803881F08238EC
:1020A00009F00BC18091EB018F708093E900809162
:1020B000EB0085FB882780F91092E90006C080912B
:1020C000E3019091E401911182609091E800977F83
:1020D0009093E8008093F1001092F100C8C0282F7F
:1020E0002D7F09F0EAC0882319F0823061F0E5C045
:1020F0008091E901813009F0E0C0933009F080E07F
:102100008093E4012BC08091E901811127C0809167
:10211000EB018F7009F4D1C08093E9002091EB00AE
:1021200020FF1CC0933021F48091EB00806214C02A
:102130009091EB0090619093EB0021E030E0A901D9
:1021400002C0440F551F8A95E2F74093EA001092AF
:10215000EA008091EB0088608093EB001092E90028
:102160008091E800877F86C08111A7C01091E901A6
:102170001F778091E3008078812B8093E30080912A
:10218000E800877F8093E8000E94420E8091E8007B
:1021900080FFFCCF8091E30080688093E300111101
:1021A00002C082E001C083E08093E60186C08058CF
:1021B000823008F082C08091E9019091EA018C3D63
:1021C00053E0950779F583E08A838AE289834FB7E4
:1021D000F894DE01139620E03EE051E2E32FF0E0B8
:1021E00050935700E49120FF03C0E295EF703F5FEA
:1021F000EF708E2F90E0EA3010F0C79601C0C096C5
:102200008D939D932F5F243149F74FBF8091E80054
:10221000877F8093E8006AE270E0CE0101960E9419
:10222000490D14C0AE014F5F5F4F6091EB010E94FA
:10223000900CBC01892B09F440C09091E800977F75
:102240009093E80089819A810E94AC0D8091E8000A
:102250008B778093E80031C0803879F58091E80071
:10226000877F8093E8008091E2018093F100809164
:10227000E8008E778093E8000E94420E1EC0811114
:102280001CC09091E9019230C0F48091E800877FF2
:102290008093E8009093E2010E94420E8091E20157
:1022A000811106C08091E30087FD02C081E001C07A
:1022B00084E08093E6010E948C0B8091E80083FF0C
:1022C0000AC08091E800877F8093E8008091EB004E
:1022D00080628093EB00AA960FB6F894DEBF0FBE23
:1022E000CDBFDF91CF911F9108950895CF93809135
:1022F000E6018823A1F0C091E900CF709091EC0035
:10230000892F817090FD80E8C82B1092E9008091A0
:10231000E80083FD0E942410CF70C093E900CF91A4
:10232000089590936B0180936A010895E0916A018A
:10233000F0916B01309721F00190F081E02D09942C
:1023400080E00895E0916A01F0916B01309721F0EF
:102350000280F381E02D09940895E0916A01F091E3
:102360006B01309721F00480F581E02D09940895E8
:1023700020916801309169018217930771F0909361
:10238000690180936801E0916A01F0916B013097D7
:1023900021F00680F781E02D0994089520916601CF
:1023A000309167018217930771F0909367018093D2
:1023B0006601E0916A01F0916B01309721F0008491
:1023C000F185E02D0994089508950C94E4110E947C
:1023D000FA1D0E94A7060C94C01ECF92DF92EF92C6
:1023E000FF920F931F93CF93DF93CDB7DEB72B9759
:1023F0000FB6F894DEBF0FBECDBF0E94BF068DE6BC
:10240000C82E81E0D82E00E010E0E02E802F0E9440
:10241000AD07F60141916F01F42EF826B1F40F5F7C
:102420001F4F0E30110589F78FEF89838A831B8236
:102430000E94031E8160782F9D838C8349815A817D
:102440006B818D810E94901240C09091CF0191FFCD
:1024500004C08B870E94B3078B8520E030E04F2DAE
:1024600050E0922FBA01022E02C0759567950A942A
:10247000E2F760FF24C02E83EF8221E030E06901A3
:1024800002C0CC0CDD1C9A95E2F790E08C219D21D6
:10249000892B09F420E028870E94031E8160782F91
:1024A0009A8789874E815F8168858A850E9490120C
:1024B000F801E359FE4F8081C826C08206C02F5F15
:1024C0003F4F2630310569F6AACF0E94A72110910F
:1024D0006C010E9496111817A1F00E94961180932A
:1024E0006C012B960FB6F894DEBF0FBECDBFDF9107
:1024F000CF911F910F91FF90EF90DF90CF900C94B0
:102500008F0A2B960FB6F894DEBF0FBECDBFDF91BA
:10251000CF911F910F91FF90EF90DF90CF90089592
:10252000CF93DF93CDB7DEB72B970FB6F894DEBF0E
:102530000FBECDBF4F83588769877A878B87DE01AF
:10254000119686E0FD0111928A95E9F785E0FE017A
:10255000379601900D928A95E1F749815A816B81F6
:102560007C818D819E810E94C0192B960FB6F894B4
:10257000DEBF0FBECDBFDF91CF9108950895CF93F9
:10258000882309F4C2C0C82F823859F40E949611DA
:1025900081FDBBC089E30E94691C0E94361D89E34E
:1025A0000CC0833879F40E94961180FDAEC083E59B
:1025B0000E94691C0E94361D83E50E94AB1CCF91CE
:1025C0000C94361D843859F40E94961182FD9DC0EA
:1025D00087E40E94691C0E94361D87E4EECF8CEFD1
:1025E0008C0F813A48F48C2F0E94EA2381118DC010
:1025F0008C2F0E94691CE3CF80E28C0F883048F456
:10260000C77081E001C0880FCA95EAF70E94EF1CED
:10261000D6CF8BE58C0F833078F4C53A29F0C63AD3
:1026200031F083E890E005C081E890E002C082E8E4
:1026300090E0CF910C94B81188E58C0F833108F0AD
:1026400064C0C83A39F1C93A41F1CA3A49F1CB3AC2
:1026500051F1CC3A59F1CD3A61F1C03B69F1CE3A32
:1026600071F1CF3A79F1C13B81F1C23B89F1C33BB2
:1026700091F1C43B99F1C53BA1F1C63BA9F1C73B20
:10268000B1F1C83BB9F1C93BC1F1CA3BC9F180E026
:1026900090E038C082EE90E035C089EE90E032C024
:1026A0008AEE90E02FC085EB90E02CC086EB90E0A6
:1026B00029C087EB90E026C08CEC90E023C08DEC25
:1026C00090E020C083E891E01DC08AE891E01AC044
:1026D00082E991E017C084E991E014C081E292E0C0
:1026E00011C083E292E00EC084E292E00BC085E26A
:1026F00092E008C086E292E005C087E292E002C064
:102700008AE292E0CF910C94CE11CF910895882364
:1027100009F44BC0823859F40E94961181FF45C0DC
:1027200089E30E94691C0E94361D89E30CC083382E
:1027300071F40E94961180FF38C083E50E94691CE5
:102740000E94361D83E50E94AB1C0C94361D843814
:1027500059F40E94961182FF28C087E40E94691CE8
:102760000E94361D87E4EFCF9CEF980F913A58F303
:1027700090E2980F983050F4877091E001C0990F63
:102780008A95EAF7892F0E94F51CDFCF9BE5980F09
:10279000933020F480E090E00C94B811885A833193
:1027A00020F480E090E00C94CE110895882321F06D
:1027B0000E94EF1C0C94361D0895882321F00E947E
:1027C000F51C0C94361D0895BF92CF92DF92EF92C4
:1027D000FF920F931F93CF93DF9300D000D000D0D0
:1027E000CDB7DEB725E0FC01DE01119601900D9218
:1027F0002A95E1F7FC01D080118102812581229583
:102800002F7043815481452B09F4FCC21F3F21F4F2
:10281000FFEFDF1609F4F6C27C012E830E94BE1280
:10282000D9821A8369817A81802F0E94651C182FB2
:10283000B92E0E941A1C0E94E11A2E81002319F061
:102840000E940C1D2E81EB2DE295EF70F0E0E05917
:10285000FF4F0C941F268B2D807F9B2D9F70F92E90
:10286000882319F0F29480EFF822002389F0FF20EA
:1028700009F475C280E2810F883020F48F2D0E9408
:10288000EF1C03C08F2D0E94FF1C0E94361D67C2E3
:10289000812F0E948713FF2009F4B4C2105E8F2D90
:1028A000183018F40E94F51C02C00E94051D2696DF
:1028B0000FB6F894DEBF0FBECDBFDF91CF911F9151
:1028C0000F91FF90EF90DF90CF90BF900C94361D4A
:1028D0003B2D307F8B2D8F70303211F08295807FB1
:1028E000112319F0113021F12CC00023B9F022235B
:1028F00009F4A0C1213009F09DC126960FB6F894C5
:10290000DEBF0FBECDBFDF91CF911F910F91FF9022
:10291000EF90DF90CF90BF900C941F1D222319F0F1
:10292000213009F46FC28E830E94221D8E8196C1D0
:10293000002321F0223008F065C27CC1211162C25F
:102940008DC1002321F0222309F474C108C222237F
:1029500009F484C119C22B2D26952695237030E0E9
:102960002115310521F021303105D1F04BC2002372
:1029700021F0812F9B2D937002C080E090E026967D
:102980000FB6F894DEBF0FBECDBFDF91CF911F9180
:102990000F91FF90EF90DF90CF90BF900C94B81103
:1029A000002321F0812F9B2D937002C080E090E0E6
:1029B00026960FB6F894DEBF0FBECDBFDF91CF9144
:1029C0001F910F91FF90EF90DF90CF90BF900C94EC
:1029D000CE11812F002319F00E94AF2002C00E9467
:1029E000172126960FB6F894DEBF0FBECDBFDF913C
:1029F000CF911F910F91FF90EF90DF90CF90BF90FC
:102A00000C949C218B2D837009F07BC00111FAC1BD
:102A1000812F829586958770880F880F912F9F70E0
:102A2000C92ED12CE12CF12C082E04C0CC0CDD1CBD
:102A3000EE1CFF1C0A94D2F714FF12C04FE050E0C6
:102A400060E070E004C0440F551F661F771F8A9531
:102A5000D2F7CB01BA01609570958095909503C02F
:102A600060E070E0CB012B2D269526952370422F38
:102A700050E042305105D9F04330510569F16C29DD
:102A80007D298E299F294130510551F126960FB697
:102A9000F894DEBF0FBECDBFDF91CF911F910F9194
:102AA000FF90EF90DF90CF90BF900C94081B6C29A3
:102AB0007D298E299F2926960FB6F894DEBF0FBE7A
:102AC000CDBFDF91CF911F910F91FF90EF90DF90DD
:102AD000CF90BF900C94241B0E94081BC701B60125
:102AE00026960FB6F894DEBF0FBECDBFDF91CF9113
:102AF0001F910F91FF90EF90DF90CF90BF900C94BB
:102B0000EC1A002319F08B2D817001C08695882363
:102B100009F478C1812F829586958770880F880F78
:102B2000912F9F70C92ED12CE12CF12C082E04C0BE
:102B3000CC0CDD1CEE1CFF1C0A94D2F714FF12C053
:102B40004FE050E060E070E004C0440F551F661F86
:102B5000771F8A95D2F7CB01BA0160957095809561
:102B6000909503C060E070E0CB012B2D2695269553
:102B70002370422F50E042305105D9F043305105C7
:102B800069F16C297D298E299F294130510551F128
:102B900026960FB6F894DEBF0FBECDBFDF91CF9162
:102BA0001F910F91FF90EF90DF90CF90BF900C940A
:102BB000E21B6C297D298E299F2926960FB6F89451
:102BC000DEBF0FBECDBFDF91CF911F910F91FF9060
:102BD000EF90DF90CF90BF900C94FE1B0E94E21B01
:102BE000C701B60126960FB6F894DEBF0FBECDBF63
:102BF000DF91CF911F910F91FF90EF90DF90CF90D9
:102C0000BF900C94C61B103FD1F118F4103E50F445
:102C1000A1C0123F09F463C008F44CC0133F09F48B
:102C200073C098C01F708B2D8F710023A1F00E947C
:102C30005F1B812F26960FB6F894DEBF0FBECDBF67
:102C4000DF91CF911F910F91FF90EF90DF90CF9088
:102C5000BF900C94D6130E94801B812F26960FB62E
:102C6000F894DEBF0FBECDBFDF91CF911F910F91C2
:102C7000FF90EF90DF90CF90BF900C94DD13002376
:102C8000A9F02111BFC08B2D8F7126960FB6F89435
:102C9000DEBF0FBECDBFDF91CF911F910F91FF908F
:102CA000EF90DF90CF90BF900C94A51B223008F0DE
:102CB000A9C0E9CF0023A9F08B2D8F7126960FB6FE
:102CC000F894DEBF0FBECDBFDF91CF911F910F9162
:102CD000FF90EF90DF90CF90BF900C945F1B00238C
:102CE00059F38B2D8F7126960FB6F894DEBF0FBE69
:102CF000CDBFDF91CF911F910F91FF90EF90DF90AB
:102D0000CF90BF900C94801B002399F08B2D8F7176
:102D100026960FB6F894DEBF0FBECDBFDF91CF91E0
:102D20001F910F91FF90EF90DF90CF90BF900C9488
:102D30004A1B26960FB6F894DEBF0FBECDBFDF91BB
:102D4000CF911F910F91FF90EF90DF90CF90BF90A8
:102D50000C94401B0023A9F0222309F4ADCF812F4E
:102D600026960FB6F894DEBF0FBECDBFDF91CF9190
:102D70001F910F91FF90EF90DF90CF90BF900C9438
:102D8000BF12222309F4ADCF812F26960FB6F894F7
:102D9000DEBF0FBECDBFDF91CF911F910F91FF908E
:102DA000EF90DF90CF90BF900C9487134B2D4F7016
:102DB000612FC7010E94420426960FB6F894DEBF29
:102DC0000FBECDBFDF91CF911F910F91FF90EF907C
:102DD000DF90CF90BF900C94641A4B2D4F70612FF1
:102DE000C70126960FB6F894DEBF0FBECDBFDF91A8
:102DF000CF911F910F91FF90EF90DF90CF90BF90F8
:102E00000C94B40726960FB6F894DEBF0FBECDBF64
:102E1000DF91CF911F910F91FF90EF90DF90CF90B6
:102E2000BF9008950E940C1D0E941C1D0E94E11C71
:102E30000E94361D0E944D220E949C2180E090E05D
:102E40000E94B81180E090E00C94CE110E94FC1C0E
:102E50000C9412170E945A1C292F22952F7030E0D3
:102E60002C3031054CF42A3031056CF422503109F4
:102E70002230310588F407C02C30310549F02F305D
:102E8000310531F009C0803E48F0803F29F406C08A
:102E900093FB882780F9089580E0089581E00895E4
:102EA000CF93DF9300D000D01F92CDB7DEB70F9045
:102EB0000F900F900F900F90DF91CF910895CF93C7
:102EC000DF9300D000D000D0CDB7DEB726960FB686
:102ED000F894DEBF0FBECDBFDF91CF9108951F9351
:102EE000CF93DF93C0917B0116E080917C01C817DE
:102EF00099F0D0E01C9FF0011D9FF00D1124E358C4
:102F0000FE4F4081518162817381848195810E944D
:102F10005F172196C770E9CFDF91CF911F91089578
:102F20004091AD015091AE016091AF017091B0013F
:102F30008091B1019091B2010C945F178091B20120
:102F400082958F7009F054C08091AF01882309F4F5
:102F50004FC080917B01A0917C016091AD01709187
:102F6000AE014091B0015091B101B6E08A1709F469
:102F70003FC090E041155105C1F17F3F11F46F3F13
:102F8000A1F1B89FF001B99FF00D1124E358FE4F55
:102F9000218172132AC02081621327C0228121114E
:102FA00024C0238134812417350710F421503109BE
:102FB000241B350B283C3105C0F42091B2012F7041
:102FC00020612093B20126E0289FF001299FF00D97
:102FD0001124EE57FE4F80818F70806180838DEACF
:102FE00091E00E94E4130C946F1701968770BECF96
:102FF0000895CF92DF92EF92FF920F931F93CF939A
:10300000DF93CDB7DEB762970FB6F894DEBF0FBE81
:10301000CDBF8C0185E0F801DE011D9601900D9277
:103020008A95E1F7D8014C9111965C91119712960F
:103030006C9112971396CD90DC9014973091AD015E
:103040007091AE018091B0019091B101009709F4A7
:103050006BC17F3F19F43F3F09F466C1E090AF01B7
:10306000EE2009F4C0C02091B201C816D90628F09C
:10307000F601E81BF90BCF0104C0809590958C0DEB
:103080009D1DFF24F394883C910578F0F12C207F5E
:1030900009F0C6C07C2DD98AC88A89890E94501738
:1030A0008DEA91E00E94E413B1C0822F807F09F085
:1030B00046C0751314C0341312C0611110C02F70B4
:1030C00020612093B2010E9490178DEA91E00E9446
:1030D000E4138091B201D80115968C932EC0CD28AF
:1030E00019F15F3F11F44F3FF9F0F62E61111CC04A
:1030F00080917B0120917C0136E0821709F45AC04F
:1031000090E0389FF001399FF00D1124E358FE4FF5
:103110007181571306C07081471303C0728171110A
:1031200003C001968770E9CFF62E662309F418C113
:103130008091B20181608093B201F12C11C17513AD
:1031400008C0341306C0611104C08091B201D801D7
:10315000C3C04D875E878D859E856A8B0E942A1726
:103160006A898823E1F16623D1F12091B201822F8F
:1031700082958F7090E0029774F08091AD019091EC
:10318000AE0198878F831986DB86CA862C87CE018D
:1031900007960E94E41386E0F801ADEAB1E00190E1
:1031A0000D928A95E1F70E949E170E949017FF24C6
:1031B000F394D6C04D875E878D859E850E945A1CEC
:1031C000292F22952F7030E0223031050CF0BCC041
:1031D0009F7009F0B6C0805E883008F4C1C0C80195
:1031E0000E94E413E4CFC816D90608F453C0F601D0
:1031F000E81BF90BCF01883C910508F450C0F12C75
:103200007C2DD98AC88A89890E945017EDEAF1E09D
:1032100086E0DF011D928A95E9F70E949017A0C011
:10322000751314C0341312C0611110C08091B20123
:10323000F8018583C8010E94E41386E0EDEAF1E01D
:10324000DF011D928A95E9F7FE2C8AC04D875E87C3
:103250008D859E856A8B0E942A176A89882309F4C6
:10326000BECF662309F4BBCF2091B201822F829595
:103270008F7090E002970CF48ECF8091AD01909109
:10328000AE019A8389831B82DD82CC822E83CE019C
:1032900001967FCF809590958C0D9D1DACCFF62E1D
:1032A000662309F49CCF75132EC034132CC02091D3
:1032B000B20120FD1FC0822F82958F70D9F0D801F6
:1032C00015962C9315978F3049F08F5F982F929514
:1032D000907F822F8F70892B15968C93C8010E9446
:1032E000E41386E0F801ADEAB1E001900D928A9511
:1032F000E1F793CF86E0F801ADEAB1E001900D92DD
:103300008A95E1F72DC04D875E878D859E850E9449
:103310002A17811140CF8091B20181608093B20160
:10332000C8010E94E4131CC0662309F458CF4D87DE
:103330005E878D859E850E942A17882309F44FCFCA
:103340002ACF811148CF0CC0243031050CF047CF73
:103350009F7009F440CFF8019581907F09F03BCF31
:103360008F2D62960FB6F894DEBF0FBECDBFDF91F2
:10337000CF911F910F91FF90EF90DF90CF90089524
:103380001F93CF93DF93CDB7DEB72C970FB6F8948A
:10339000DEBF0FBECDBF4F83588769877A878B8783
:1033A0009C87CE0107960E94F917882369F08F81C8
:1033B00098852A853B85232BF1F19F3F09F063C057
:1033C0008F3F09F060C037C086E0FE013796DE010E
:1033D000119601900D928A95E1F76F817885EA85C3
:1033E000FB85309741F17F3F11F46F3F21F1209130
:1033F0007C0130E0C90101968770992740917B01DB
:1034000050E08417950709F447C069837A83FD83E8
:10341000EC8396E0929FD001939FB00D1124A358A6
:10342000BE4FFE01319601900D929A95E1F780937F
:103430007C010E946F1716E080917B0190917C01C6
:103440008917C1F1189FC001112483589E4F0E9413
:10345000F917882379F1E0917B011E9FF001112477
:10346000E358FE4F4081518162817381848195814F
:103470000E945F1780917B0190E0019687709927E9
:1034800080937B01D9CF4F81588569857A858B855B
:103490009C850E945F17CFCF0E94261710927C0157
:1034A00010927B01EDEAF1E086E0DF011D928A9542
:1034B000E9F7C1CF2C960FB6F894DEBF0FBECDBF93
:1034C000DF91CF911F910895EF92FF920F931F9379
:1034D000CF93DF938C01892B09F46CC0F12CEE247F
:1034E000E394E8012196F8018491843740F4843014
:1034F00008F051C0813081F0823019F15BC085370E
:1035000009F444C0A8F19CE7980F903708F052C026
:103510008F770E94871341C00E5F1F4FFE01C49139
:1035200080E28C0F883048F4C7708E2D01C0880F60
:10353000CA95EAF70E940F1D14C08C2F0E94BF127B
:103540002DC00E5F1F4FFE01C49180E28C0F8830AA
:1035500058F4C7708E2D01C0880FCA95EAF70E94F3
:10356000151D0E94361D1AC08C2F0E94871316C08D
:103570000E5F1F4FFE01C491CC2381F08FE99FE0C5
:103580000197F1F700C00000C150F6CF0E5F1F4F4A
:10359000FE01F49003C00E94BF128E018F2D88237C
:1035A00009F49FCFEFE9FFE03197F1F700C0000089
:1035B0008150F5CFDF91CF911F910F91FF90EF9048
:1035C000089508956093B7017093B8018093B9018D
:1035D0009093BA010C9412170F931F930091B701A7
:1035E0001091B8012091B9013091BA01DC01CB01F1
:1035F000802B912BA22BB32B8093B7019093B80112
:10360000A093B901B093BA011F910F910C941217B6
:103610000F931F930091B7011091B8012091B90148
:103620003091BA01DC01CB0180239123A223B32383
:103630008093B7019093B801A093B901B093BA01F8
:103640001F910F910C9412170F931F930091B701C4
:103650001091B8012091B9013091BA01DC01CB0180
:1036600080279127A227B3278093B7019093B801B1
:10367000A093B901B093BA011F910F910C94121746
:103680001092B3011092B4011092B5011092B601DC
:103690000C94121741E050E060E070E004C0440F69
:1036A000551F661F771F8A95D2F74093B301509339
:1036B000B4016093B5017093B6010C94121741E008
:1036C00050E060E070E004C0440F551F661F771F94
:1036D0008A95D2F78091B3019091B401A091B50180
:1036E000B091B601482B592B6A2B7B2B4093B30129
:1036F0005093B4016093B5017093B6010C94121706
:1037000041E050E060E070E004C0440F551F661FC8
:10371000771F8A95D2F74095509560957095809166
:10372000B3019091B401A091B501B091B6014823C5
:1037300059236A237B234093B3015093B4016093D0
:10374000B5017093B6010C94121741E050E060E0AF
:1037500070E004C0440F551F661F771F8A95D2F78B
:103760008091B3019091B401A091B501B091B601DF
:10377000482759276A277B274093B3015093B40108
:103780006093B5017093B6010C9412170F931F93B9
:103790000091B3011091B4012091B5013091B601AF
:1037A000DC01CB01802B912BA22BB32B8093B30197
:1037B0009093B401A093B501B093B6011F910F91FE
:1037C0000C9412170F931F930091B3011091B40141
:1037D0002091B5013091B601DC01CB01802391230A
:1037E000A223B3238093B3019093B401A093B501B6
:1037F000B093B6011F910F910C9412170F931F9362
:103800000091B3011091B4012091B5013091B6013E
:10381000DC01CB0180279127A227B3278093B30136
:103820009093B401A093B501B093B6011F910F918D
:103830000C9412170895CF92DF92EF92FF920F939C
:103840001F93CF93DF938C01C090B701D090B80144
:10385000E090B901F090BA018091B3019091B40168
:10386000A091B501B091B601C82AD92AEA2AFB2A4B
:10387000CFE1D0E0D701C6010C2E04C0B695A795C4
:10388000979587950A94D2F780FF06C0B8018C2FD0
:103890000E94F409019721F4219760F780E001C0AC
:1038A0008C2FDF91CF911F910F91FF90EF90DF90C0
:1038B000CF900895CF93DF93EC010E941B1CBE01B3
:1038C0000E94F409DF91CF910895CB010E945A1C08
:1038D000089590910C01992321F090910D0191117F
:1038E00009C020910E0130910F01F90132969FEF2E
:1038F00040E01FC0982F9695969596959F3050F56D
:10390000E0910E01F0910F01E90FF11D877021E0A8
:1039100030E0A90102C0440F551F8A95E2F7CA01A1
:103920009181892B818308959F3F39F04F5F4E30FD
:1039300041F051915813F8CF0DC05111F7CF942F8A
:10394000F5CF9F3F39F0F901E90FF11D97FDFA9589
:1039500082830895089590910C01992321F090910C
:103960000D01911109C020910E0130910F01F90153
:103970003296205F3F4F1FC0982F9695969596954B
:103980009F30F0F4E0910E01F0910F01E90FF11D6D
:10399000877021E030E0A90102C0440F551F8A95CD
:1039A000E2F7CA0180959181892381830895319638
:1039B000E217F30729F090819813F9CF1082F7CF1F
:1039C000089581E090E0E0910E01F0910F01E80F81
:1039D000F91F1082019680319105A9F70895909101
:1039E000CE01892B8093CE01089580959091CE01D0
:1039F00089238093CE0108951092CE01089590916D
:103A0000CD01892B8093CD01089580959091CD01B2
:103A100089238093CD0108951092CD01089590914E
:103A2000CC01892B8093CC01089580959091CC0195
:103A300089238093CC0108951092CC01089580933E
:103A4000BB0108951092BB01089580910E019091E1
:103A50000F01FC0131969C01205F3F4F80E0919166
:103A600091118F5FE217F307D1F70895E0910E01EE
:103A7000F0910F018091CE018083E0910E01F091D1
:103A80000F0190818091CD01892B8083E0910E01FF
:103A9000F0910F0190818091CC01892B80838091DE
:103AA000BB01882361F0E0910E01F0910F0190813C
:103AB000892B80830E94251D81111092BB0180916A
:103AC0000E0190910F010C94A211CF92DF92EF9210
:103AD000FF926C01EE24FF24C114D104E104F1042F
:103AE00021F0C701B60120E101C020E0C72ED82E89
:103AF000E92EFF24C114D104E104F10419F0285F78
:103B0000C701B6016B017C0154E0F694E794D794A9
:103B1000C7945A95D1F7C114D104E104F10419F006
:103B20002C5FC701B6016B017C0142E0F694E7947B
:103B3000D794C7944A95D1F7C114D104E104F10494
:103B400019F02E5FC701B601DC01CB01B695A79530
:103B500097958795892B8A2B8B2B09F02F5F822FC6
:103B6000FF90EF90DF90CF9008958091E601843030
:103B700021F11092D00120E488E190E00FB6F89492
:103B8000A895809360000FBE2093600080E00E94A3
:103B90008F0A83B7817F846083BF83B7816083BFCF
:103BA0007894889583B78E7F83BF88E10FB6F894A9
:103BB00080936000109260000FBE089508950895EC
:103BC000CF930E94DE1D0E94BF060E94DF1DC0E051
:103BD0008C2F0E94AD07811104C0CF5FCE30C1F79A
:103BE00001C081E0CF9108950E9426170E9496118E
:103BF0000C948F0A82E084BD93E095BD9AEF97BD47
:103C000080936E0008952FB7F8948091D101909120
:103C1000D201A091D301B091D4012FBF0895CF92CA
:103C2000DF92EF92FF920F931F932FB7F89440917A
:103C3000D1015091D2016091D3017091D4012FBF75
:103C40006A017B01EE24FF248C0120E030E0C016E5
:103C5000D106E206F30610F4415051099A01281BDF
:103C6000390BC9011F910F91FF90EF90DF90CF901A
:103C700008951F920F920FB60F9211248F939F9366
:103C8000AF93BF938091D1019091D201A091D301C4
:103C9000B091D4010196A11DB11D8093D1019093E3
:103CA000D201A093D301B093D401BF91AF919F9162
:103CB0008F910F900FBE0F901F9018950E94930E3A
:103CC000F8942FEF87EA91E6215080409040E1F789
:103CD00000C0000087E090EBDC018093F00190933E
:103CE000F101A093F201B093F3019CE088E10FB6DB
:103CF000F894A895809360000FBE90936000FFCF6A
:103D0000EF92FF920F931F93CF93DF93D82FC0E0D2
:103D10008C2F0E94AD0700E010E0E82EF12CC701C7
:103D2000002E02C0959587950A94E2F780FD06C0A3
:103D30000F5F1F4F0630110591F709C0602F7C2FD0
:103D400080E00E94B507D813F3CF81E004C0CF5FB5
:103D5000CE30F1F680E0DF91CF911F910F91FF906F
:103D6000EF900895CF93C82F8CE20E94801E882385
:103D700021F08C2FCF910C94801E80E0CF9108957C
:103D8000CF930E940720811102C00E94ED1FC5E65B
:103D9000C15049F00E94BF068FE39CE90197F1F7FB
:103DA00000C00000F5CF89E20E94B21E811113C14C
:103DB0008AE20E94B21E81110E94ED1F85E00E94DE
:103DC000B21E81110E945E1E0E9412208093CF01BC
:103DD00087E00E94B21E8823A9F18BE10E94B21EE7
:103DE000882351F08091CF0181FB222720F991E0B7
:103DF000922790FB81F90EC08EE00E94B21E8823AC
:103E000061F08091CF0182FB222720F991E0922777
:103E100090FB82F98093CF0115C080E10E94B21E11
:103E20009091CF01882341F093FB222720F981E074
:103E3000822780FB93F904C0892F809580FB90F93D
:103E40009093CF018091CF010E9416200E942420E0
:103E50008093EF0180EE0E94B21E882341F0809192
:103E6000EF01982F909590FB80F98093EF0189E303
:103E70000E94B21E882359F08091EF0181FB222716
:103E800020F991E0922790FB81F98093EF0182EE77
:103E90000E94B21E882359F08091EF0182FB2227F5
:103EA00020F991E0922790FB82F98093EF0186EE52
:103EB0000E94B21E882359F08091EF0183FB2227D4
:103EC00020F991E0922790FB83F98093EF0183EE34
:103ED0000E94B21E882359F08091EF0184FB2227B3
:103EE00020F991E0922790FB84F98093EF0185E31C
:103EF0000E94B21E882359F08091EF0185FB222792
:103F000020F991E0922790FB85F98093EF0181E3FE
:103F10000E94B21E882359F08091EF0186FB222770
:103F200020F991E0922790FB86F98093EF0181E1DF
:103F30000E94B21E882359F08091EF0187FB22274F
:103F400020F991E0922790FB87F98093EF0180910F
:103F5000EF010E9428208091EF0187FB882780F9DC
:103F600080930D0187E20E94B21EC82F8EE10E944D
:103F7000B21E8111C2608FE10E94B21E8111C46025
:103F800080E20E94B21E8111C86081E20E94B21ECE
:103F90008111C06182E20E94B21E8111C06283E27F
:103FA0000E94B21E8111C06484E20E94B21E882366
:103FB00011F0C06802C0CC2329F08C2F0E941F2072
:103FC0006C2F03C00E941B20682F70E080E090E0FF
:103FD000CF910C94E21ACF9108956DEE7EEF80E0C0
:103FE00090E00E94552660E082E090E00E94472623
:103FF00060E083E090E00E94472660E084E090E08B
:104000000E94472660E085E090E00C94472680E01F
:1040100090E00E94412621E08D3E9E4F09F020E075
:10402000822F089582E090E00C943926682F82E078
:1040300090E00C94472683E090E00C943926682F9A
:1040400083E090E00C94472684E090E00C943926BD
:10405000682F84E090E00C9447268091D70180FF80
:104060000BC06091130185E0689FB0011124759524
:104070006795759567952BC081FF09C06091130105
:1040800085E0689FB00111247595679520C082FF77
:1040900007C06091130185E0689FB001112417C02B
:1040A0009091D8019923D1F060911201961788F769
:1040B0002091130185E0289F90011124929FA00177
:1040C000939F500D112470E0CA010E940B266038A6
:1040D000710540F46115710539F002C065E070E0CA
:1040E000862F08958FE7089581E008958091D70184
:1040F00080FF08C06091110170E075956795759516
:10410000679521C081FF06C06091110170E075952F
:10411000679519C082FF04C06091110170E010C062
:104120009091D8019923C1F0609110019617A0F7E2
:1041300080911101899FC001112470E00E940B261B
:104140006038710528F46115710521F0862F0895F6
:104150008FE7089581E0089561E070E0F4CF803F3B
:1041600021F40E942D20819504C0813F29F40E94F2
:104170002D208093DB010895823F21F40E942D20A1
:10418000819504C0833F29F40E942D208093DA0199
:104190000895893F19F40E94762005C08A3F31F4C2
:1041A0000E94762081958093DC0108958B3F21F455
:1041B0000E947620819504C08C3F29F40E947620CD
:1041C0008093DD010895843F21F48091D9018160BD
:1041D00017C0853F21F48091D901826011C0863FCC
:1041E00021F48091D90184600BC0873F21F4809134
:1041F000D901886005C0883F31F48091D901806180
:104200008093D90108958D3F21F48091D701816079
:104210000BC08E3F21F48091D701826005C08F3F93
:1042200029F48091D70184608093D7010895803F5D
:1042300039F48091DB0187FF6CC01092DB0169C00B
:10424000813F29F48091DB011816BCF362C0909184
:10425000DA01823F29F497FF5CC01092DA0159C05D
:10426000833F19F41916CCF354C0893F41F480916F
:10427000DC0118160CF04DC01092DC014AC08A3FD8
:1042800029F48091DC0187FF44C0F6CF8B3F39F4DD
:104290008091DD0187FF3DC01092DD013AC08C3F67
:1042A00029F48091DD011816BCF333C0843F21F45A
:1042B0008091D9018E7F17C0853F21F48091D9016B
:1042C0008D7F11C0863F21F48091D9018B7F0BC077
:1042D000873F21F48091D901877F05C0883F31F461
:1042E0008091D9018F7E8093D90113C08D3F21F435
:1042F0008091D7018E7F0BC08E3F21F48091D70132
:104300008D7F05C08F3F29F48091D7018B7F8093EB
:10431000D7018091DA0181110EC08091DB018111FA
:104320000AC08091DC01811106C08091DD018111FC
:1043300002C01092D801089589ED91E00E94AD115C
:104340000E94031E9093D6018093D50108951F9378
:10435000CF93DF938091D5019091D6010E940F1EDB
:10436000AC019091D801992321F02091140130E003
:1043700006C0209115018AE0289F90011124421760
:10438000530708F486C08091DA01C091DB01D09117
:10439000DC011091DD01811107C0C11176C0D1117E
:1043A00074C0111172C075C09F3F19F09F5F909348
:1043B000D801181624F40E942D208093DA018091F0
:1043C000DA0187FF05C00E942D2081958093DA01D4
:1043D0001C1624F40E942D208093DB018091DB01C8
:1043E00087FF05C00E942D2081958093DB0160919D
:1043F000DA01662339F1C091DB01CC2319F177276B
:1044000067FD7095872F972F0E941C2523E333E3C8
:1044100043E35FE30E9480250E94E9246093DA0170
:104420006C2F772767FD7095872F972F0E941C258B
:1044300023E333E343E35FE30E9480250E94E92402
:104440006093DB011D1624F40E9476208093DC012A
:104450008091DC0187FF05C00E94762081958093C2
:10446000DC01111624F40E9476208093DD018091F6
:10447000DD0187FF05C00E94762081958093DD01D4
:10448000DF91CF911F910C949C219F3F09F08ECF1B
:1044900096CFDF91CF911F910895E9EDF1E085E08E
:1044A000DF011D928A95E9F71092D8011092D70189
:1044B0000895833081F128F4813059F08230D1F0B1
:1044C0000895853009F449C0B8F1863009F456C022
:1044D000089580911501262F30E0280F311D2F3FC0
:1044E000310524F4680F6093150108958FEF8093D0
:1044F0001501089580911401262F30E0280F311DF9
:104500002F3F310524F4680F6093140108958FEF55
:1045100080931401089580911301262F30E0280F15
:10452000311D2F3F310524F4680F60931301089566
:104530008FEF80931301089580911201262F30E0B0
:10454000280F311D2F3F310524F4680F60931201AD
:1045500008958FEF80931201089580911101262F05
:1045600030E0280F311D2F3F310524F4680F609390
:10457000110108958FEF809311010895809110012A
:10458000262F30E0280F311D2F3F310524F4680F0E
:104590006093100108958FEF809310010895833088
:1045A00011F128F4813049F0823091F0089585307E
:1045B00081F120F18630C1F10895809115016817CD
:1045C00020F4861B8093150108951092150108951B
:1045D00080911401681720F4861B809314010895BC
:1045E00010921401089580911301681720F4861B1E
:1045F0008093130108951092130108958091120180
:10460000681720F4861B80931201089510921201FE
:10461000089580911101681720F4861B8093110181
:10462000089510921101089580911001681720F4E7
:10463000861B8093100108951092100108950F9326
:104640001F938D3109F46BC008F03FC08E3009F420
:104650007FC0C0F4873009F469C068F4863009F07F
:10466000B1C08091CF01817F8E7F8093CF0181E0A7
:104670008093DF01A8C0883009F4A2C08B3009F410
:104680009FC0A0C0863109F49BC078F4803109F442
:1046900072C0813109F096C00E94261790910D01D9
:1046A00081E0892780930D018BC0893109F488C08E
:1046B0008B3109F087C08091CF0181FB222720F93F
:1046C00091E0922790FB81F94CC0853309F470C0CA
:1046D00048F4873209F46CC008F459C0893209F4EF
:1046E00067C070C0833438F48A3308F04EC0883312
:1046F00009F466C067C0833409F45AC0883409F0ED
:1047000061C00E9426170FEF13ED20E30150104007
:104710002040E1F700C000000E945E1E51C00E94D0
:10472000A3240E9496110E948F0A4AC09091CF0143
:10473000892F8095817080FB90F929F096609860B0
:104740009093CF0140C0997F977F9093CF0138C05D
:104750008091CF0182FB222720F991E0922790FBE4
:1047600082F98093CF01992359F18091CF01816023
:104770008093CF0125C08091CF0183FB222720F9B0
:1047800091E0922790FB83F9ECCF895301C08D51C2
:1047900041E050E060E070E08A019B0104C0000F3E
:1047A000111F221F331F8A95D2F7C901B80104C017
:1047B00061E070E080E090E00E94E21A0E9426171B
:1047C00081E001C080E01F910F91089580E008957D
:1047D00080E00895CF93C82F8091DF01813079F078
:1047E00018F08230E9F187C0E0910E01F0910F01DD
:1047F0008081813169F0823209F07FC009C0E09187
:104800000E01F0910F018081813111F0823261F44B
:104810008C2F0E94E623811104C08C2F0E941F233D
:104820001DC081E090E01AC08C2F0E94E823811106
:1048300014C0C43179F048F4CB3079F0C03109F0BC
:1048400060C082E08093DF0108C0C93219F0C8332C
:1048500021F057C01092DF0154C081E0817053C035
:10486000C93289F118F5C43171F1A8F4C73009F0E3
:1048700046C08AE08093150194E19093140193E07F
:10488000909313018093120188E08093110188E2D4
:104890008093100134C0CE51C63088F5EC2FF0E083
:1048A000E65DFE4F80818093DE0129C0CE34E9F0C1
:1048B00020F4CB3421F56AE013C0C13579F0C2355C
:1048C000F1F461E00DC08091DE01882319F01092AF
:1048D000DE0115C081E08093DF0115C061E006C0F4
:1048E0008091DE010E9459220AC06AE08091DE01B7
:1048F0000E94CF2204C01092DF0180E004C081E05A
:1049000002C080E0ABCFCF910895E1E8F0E0808174
:10491000886080838081816080838FB7F89493E082
:104920009093890090ED909388008FBF0895EFE6F3
:10493000F0E08081826080830895EFE6F0E080817E
:104940008D7F80830895EFE6F0E0908182E08927F3
:10495000808308951F920F920FB60F9211242F9308
:104960003F934F935F936F937F938F939F93AF93F7
:10497000BF93EF93FF938091E0019091E101019645
:104980009093E1018093E001811103C082E00E94D5
:104990008F0AE091E101E695E695F0E0E854F84FE2
:1049A000E4918091E0018E1303C080E00E948F0AA1
:1049B000FF91EF91BF91AF919F918F917F916F91F7
:1049C0005F914F913F912F910F900FBE0F901F90CD
:1049D000189504D06894B1118DC0089570D088F0F6
:1049E0009F5790F0B92F9927B751A0F0D1F0660FDB
:1049F000771F881F991F1AF0BA95C9F712C0B130F6
:104A000081F077D0B1E0089574C0672F782F8827A0
:104A1000B85F39F0B93FCCF3869577956795B39534
:104A2000D9F73EF490958095709561957F4F8F4FA3
:104A30009F4F0895E89409C097FB3EF490958095A8
:104A4000709561957F4F8F4F9F4F9923A9F0F92F54
:104A500096E9BB279395F695879577956795B795D2
:104A6000F111F8CFFAF4BB0F11F460FF1BC06F5FB8
:104A70007F4F8F4F9F4F16C0882311F096E911C0CA
:104A8000772321F09EE8872F762F05C0662371F0EB
:104A900096E8862F70E060E02AF09A95660F771FFF
:104AA000881FDAF7880F9695879597F9089557FD2F
:104AB0009058440F551F59F05F3F71F04795880F8C
:104AC00097FB991F61F09F3F79F087950895121623
:104AD00013061406551FF2CF4695F1DF08C01616CF
:104AE00017061806991FF1CF869571056105089480
:104AF0000895E894BB2766277727CB0197F9089597
:104B00000BD078C069D028F06ED018F0952309F04A
:104B10005AC05FC01124EECFCADFA0F3959FD1F336
:104B2000950F50E0551F629FF001729FBB27F00D5B
:104B3000B11D639FAA27F00DB11DAA1F649F6627B0
:104B4000B00DA11D661F829F2227B00DA11D621FFF
:104B5000739FB00DA11D621F839FA00D611D221FB9
:104B6000749F3327A00D611D231F849F600D211D9D
:104B7000822F762F6A2F11249F5750408AF0E1F040
:104B800088234AF0EE0FFF1FBB1F661F771F881F89
:104B900091505040A9F79E3F510570F014C0AACF24
:104BA0005F3FECF3983EDCF3869577956795B79574
:104BB000F795E7959F5FC1F7FE2B880F911D96959E
:104BC000879597F9089597F99F6780E870E060E00E
:104BD00008959FEF80EC089500240A941616170696
:104BE00018060906089500240A94121613061406DE
:104BF00005060895092E0394000C11F4882352F041
:104C0000BB0F40F4BF2B11F460FF04C06F5F7F4FF8
:104C10008F4F9F4F089597FB072E16F4009407D0EF
:104C200077FD09D00E94252607FC05D03EF490951B
:104C300081959F4F0895709561957F4F0895EE0F70
:104C4000FF1F0590F491E02D0994AA1BBB1B51E1B5
:104C500007C0AA1FBB1FA617B70710F0A61BB70BEC
:104C6000881F991F5A95A9F780959095BC01CD0191
:104C70000895F999FECF92BD81BDF89A992780B524
:104C80000895A8E1B0E042E050E00C945C26262FA5
:104C9000F999FECF1FBA92BD81BD20BD0FB6F89421
:104CA000FA9AF99A0FBE019608950E944726272F77
:104CB0000C944826DC01CB01FC01F999FECF06C01B
:104CC000F2BDE1BDF89A319600B40D9241505040CA
:084CD000B8F70895F894FFCF36
:104CD8002002910A1F0BFC0AC80A940A0101BC01B0
:104CE80028080A03140A3F4D363979072C07F606B7
:104CF800BD065006690682069B06010203040506E6
:044D0800070809008F
:00000001FF
